:020000003B289B
:06000A009D006E309E0017
:100010000000000000000000000000009E0B082807
:100020009D0B062800349101900A10080A3A031922
:10003000900108009201910A11080A3A031913204D
:1000400008009301920A12080A3A03191A200800BC
:10005000930A13080A3A03192120FA3005200800F0
:1000600082073F34183476347C3459346D346F341D
:1000700038347F347D34831610308500003086009C
:100080008312900191019201930100308500051EB9
:10009000282008308F0010308400003086000F08C0
:1000A0008500000830208600033005200F184728FF
:0800B00003108F0C840A4D2897
:00000001FF
